:020000001828BE
:080008008E00030E8D0083162B
:100010008B1C1028831286185C288B100B168316F5
:100020000B184F2083120D0E83008E0E0E0E09004A
:1000300083128B1308308900831608148312000082
:100040000808081E3428003089000310153E84007B
:100050000830A300831608148312000008088000EB
:10006000840A890AA30B2A28831601138113061612
:1000700086160617861406148312003092000B10A1
:100080008B100B168B158B17060870398C0003101C
:100090008C0C8C0C8C0C30308C074F204E2883122B
:1000A000060870398C0003108C0C8C0C8C0C3030D2
:1000B0008C070B108B1508008312382112100F18B3
:1000C00012140F100F0803110C06031D7028642171
:1000D000121872289A2883128B100B168316102878
:1000E00072216B28382164210F089300931981280D
:1000F000073013050310153E8400000890004C21C2
:100100006B28423090004C21613090004C217330BC
:1001100090004C21653090004C21203090004C2103
:10012000313090004C212E3090004C213030900026
:100130004C216B28382164210F0893003821642159
:100140000F089400E03013059200003003111206EE
:100150000319C728203012060319CF284030120691
:100160000319D928603012060319EE2880301206D0
:1001700003190829A030120603191429C0301206E9
:1001800003192529E0301206031937296B28073097
:1001900013050310153E8400140880006B281530E9
:1001A00084000830910014088000840A910BD32841
:1001B0006B280730130589000310153E84000008E2
:1001C00088008316081555308900AA3089008814E4
:1001D0000811081EE928081283126B2800308900D4
:1001E0000310153E84000830910000088800831633
:1001F000081555308900AA30890088140811081E96
:10020000FF2808128312890A840A910BF5286B28AB
:100210000730130589000310153E84008316081467
:100220008312080880006B28003089000310153EF7
:100230008400083091008316081483120808800097
:10024000840A890A910B1B296B2808308900103019
:10025000130588008316081555308900AA308900D7
:1002600088140811081E3229081283126B286B2883
:100270008F010830910086183B29861C3D29061CF9
:100280004229452903108F0D492903108F0D0F14A2
:100290004929910B3B29080008309100831606106C
:1002A000831286185129861C5329900D031C592945
:1002B0005B2906105D2906145D29910B51297221D5
:1002C000831606148312080086186429861C662982
:1002D000061083160610831286186C2983160614DE
:1002E0008312080086187229861C742986187629BC
:0202F000080004
:00000001FF
